:100000000C942A001895000018950000189500001F
:10001000189500001895000018950000189500002C
:10002000189500000C94D10918950000189500004F
:10003000189500001895000018950000189500000C
:1000400018950000189500001895000018950000FC
:10005000189500008FE58DBFC4E0E0E84E2E88E0E3
:100060008EBFD8E0F7E05F2EEEEFF7E0A0E6B0E05D
:1000700088278D933197E9F783E389B980E080BDC4
:1000800088E18AB9662487E08ABB87EF8BBB8FEB58
:1000900087BB8FEB88BB80EE84BB8FEF85BB80E88E
:1000A00081BB8BE382BB80E08FBD81E08EBD8FE1A1
:1000B00081BD87E181BD86E086B980E487B9C398B8
:1000C000C29AD89AC498C798C598F894A895809170
:1000D0006B008F7D80936B000027ABE6B0E08C91C6
:1000E00085FB0EF401E041E0041711F00C947C0054
:1000F00087E88ABB87E78BBB0E942B0B8091D100DE
:1001000088608093D100EFEFF1E0A2ECB0E091E0E5
:100110000E94E8240091C200003081E009F080E0F4
:100120008F930091C2000E3F80E010F009F081E053
:100130009F91892B882311F40C94A1008EEB80935E
:10014000C2000091C2004AE0040F01BF82E390E0C8
:100150000E94A723E6E2FAE40E940B23ABE6B0E09C
:100160008C9185FBA8E6B7E00E94FF238D9388273A
:100170008C930E9403230E941723EAE0F0E0BB2740
:10018000A0E10E94E5240D3311F40C94FD00EBE096
:10019000F0E0A0E1BB2788E08C937BE70E94D424A9
:1001A000ECE0F0E001E010E0A0E1BB277BE70E947B
:1001B000D624EAE0F0E0A0E1BB278DE38C937BE757
:1001C0000E94D424EEE0F0E0A0E1BB2780E08C9315
:1001D0007BE70E94D424E0E1F0E000E010E0A0E141
:1001E000BB277BE70E94D624EFE0F0E0A0E1BB272D
:1001F00080E08C937BE70E94D424EBE0F0E0ADEB51
:10020000B0E00E94E5240091BD000C3318F011F01D
:100210000C940C010C940F018CE38093BD0080E7DB
:1002200097E9AEEBB0E08D939C93ECE0F0E0A8EBA7
:10023000B0E00E94E724EEE0F0E0A3ECB0E00E9422
:10024000E524EFE0F0E0A4ECB0E00E94E5240E9499
:100250002F0BE0E1F0E0A4E6B0E00E94E724A4E682
:10026000B0E00E949522E0E1F0E0A4E6B0E07BE798
:100270000E94D624A8EBB0E00D911C91003050E014
:10028000150711F00C944A0181E090E0A8EBB0E072
:100290008D939C93EEE3FAE40E940B23A8E6B7E06B
:1002A000EDEBF0E00E946D240E940323E6E4FAE403
:1002B0000E940B23A8E6B7E0E8EBF0E00E945E2482
:1002C0000E940323E6E4FAE40E940B23A8E6B7E0C9
:1002D000E3ECF0E00E946D240E940323E6E4FAE4DC
:1002E0000E940B23A8E6B7E0E4ECF0E00E946D2446
:1002F0000E940323E6E4FAE40E940B23A8E6B7E099
:10030000E4E6F0E00E945E240E940323E6E4FAE4BF
:100310000E940B23BB27A3E38C9180FBA8E6B7E0E8
:100320000E94FF238D9388278C930E9403230E94B1
:1003300017230027BB27A3E38C9180FB0EF401E079
:1003400041E0041711F00C94B10180916B008B7F98
:1003500080936B00A3ECB0E08C918E7F8C930C9417
:10036000BB0180916B00846080936B00A3ECB0E0D4
:100370008C9181608C9380916B008B7F80936B005C
:10038000A3ECB0E08C918E7F8C938091D1008F7D17
:100390008093D100A3ECB0E08C918D7F8C93809101
:1003A0006B008F7B80936B0080E882BB979880E026
:1003B0008093D00080916B008D7F80936B0080E0F4
:1003C0008093C60086E08093C0008DE08093C100DA
:1003D00084E190E00E94A7230E949323C49AE8E45A
:1003E000FAE40E940B230E94172388EC90E00E94FD
:1003F000A723A89581B5886181BD877F81BDE0E68F
:10040000F0E0FA93EA930E9412182296A8950091C0
:100410006000003011F40C9419020E945417E2E5B8
:10042000FAE40E940B230E9417230E94F50A0C9401
:100430001E028091D1008F7E8093D100ECE5FAE41A
:100440000E940B230E947D1784E690E00E94A72360
:100450000027A1EDB0E08C9184FB0EF401E040E0B8
:10046000041711F00C9436020E94110E8FEF0E94B7
:100470001A2382E390E00E94A7237894A89581B57F
:10048000886081BDA4EBB0E04D915C91A8EBB0E039
:100490000D911C910417150718F011F00C945202DD
:1004A0000C94580281E090E0A8EBB0E08D939C930F
:1004B00080E08093BA0080E080936A0080E08093BF
:1004C0006C000027A1EDB0E08C9184FB0EF401E0FC
:1004D00041E0041711F00C946F020E942B0BA895B9
:1004E0000E94FB22ADE6B0E08D9388278C93E3E673
:1004F000F0E0FA93EA930E94D616229600916300E8
:10050000003081E009F080E08F930091D00001304D
:1005100081E009F080E09F918923882311F40C94F5
:1005200093020E94D90A81E090E00E94A7230091E3
:10053000D000003081E009F080E08F930027ABE627
:10054000B0E08C9181FB0EF401E041E0041781E002
:1005500009F080E09F91892B882311F40C94B40258
:1005600085E090E00E94A7230027BB27A3E38C919E
:1005700082FB0EF401E040E0041711F00C94F40249
:100580000091BD00023018F011F00C94C9020C94D7
:10059000F002ADEBB0E08C9182508C938EB5887FE9
:1005A0008EBD5A924A928091BD00A42DB52D8C9398
:1005B00081E00E9482220E94001F229681E00E9418
:1005C0007E22EBE0F0E0ADEBB0E07BE70E94D424CC
:1005D0000091D000013011F00C94F00281E08EBD4A
:1005E00084E690E00E94A7230027BB27A3E38C9119
:1005F00083FB0EF401E040E0041711F00C9431038A
:100600000091BD00063410F00C942D03ADEBB0E06A
:100610008C918E5F8C938EB5887F8EBD5A924A9254
:100620008091BD00A42DB52D8C9381E00E94822283
:100630000E94001F229681E00E947E22EBE0F0E003
:10064000ADEBB0E07BE70E94D4240091D0000130F4
:1006500011F00C942D0381E08EBD84E690E00E94A1
:10066000A723ADE6B0E08C91803081E009F480E012
:100670008F9340916C0000916300041781E009F4AE
:1006800080E09F91892B8F930091BA00013081E027
:1006900009F080E09F91892B882311F40C9461026A
:1006A0008091630080936C0000916300003081E0D2
:1006B00009F480E08F930091BA00003081E009F0E6
:1006C00080E09F918923882311F40C94D8038EB580
:1006D000887F8EBD8AE090E00E94A723E3E6F0E0E9
:1006E000FA93EA930E94D616229600916300003096
:1006F00011F40C94A703A3E6B0E08C91A8EBB0E052
:100700008D9388278C9300916300043011F00C9432
:100710008F0383E090E0A8EBB0E08D939C93009171
:100720006300083011F00C949B0384E090E0A8EB88
:10073000B0E08D939C9300916300003111F00C9414
:10074000A70385E090E0A8EBB0E08D939C93A4EB29
:10075000B0E04D915C91A8EBB0E00D911C910417B5
:10076000150780E010F009F081E08F93A8EBB0E06E
:100770000D911C91003050E0150781E009F080E0F8
:100780009F91892B882311F40C94CC0381E090E095
:10079000A8EBB0E08D939C9300916300003011F4BE
:1007A0000C94D803ADE6B0E0E6E6FAE40E94E92353
:1007B000EDE6F0E0ADE6B0E00E94F3230091BA0070
:1007C000013011F00C94FF0380E08093BA00ADE695
:1007D000B0E0E8E6FAE40E94E9230027BB27A3E3A0
:1007E0008C9181FB0EF401E040E0041711F00C94B1
:1007F000FF03ADE6B0E0E6E6FAE40E94E923ADE6E9
:10080000B0E0EAE6FAE40E94FF2411F00C944604FA
:100810005A924A928091C000A42DB52D8C9381E00C
:100820000E9482225A924A928091C100A42DB52D35
:100830008C9381E00E9482220E94591F249682E0BC
:100840000E947E220091C40041E0042BA0E6B0E0AB
:100850000C938091D10084608093D1008EB5887F05
:100860008EBDEFE0F0E0A0E6B0E07BE70E94D4248C
:10087000809160008093C4000091D000013011F09D
:100880000C94440481E08EBD0C94CB09ECE6FAE4B0
:100890000E94FF2411F00C9489045A924A9280E03D
:1008A000A42DB52D8C9381E00E9482225A924A9207
:1008B00080E0A42DB52D8C9381E00E9482220E94BD
:1008C000591F249682E00E947E220091C4004EEFC0
:1008D0000423A0E6B0E00C938091D1008B7F80933D
:1008E000D1008EB5887F8EBDEFE0F0E0A0E6B0E0ED
:1008F0007BE70E94D424809160008093C400009123
:10090000D000013011F00C94870481E08EBD0C946E
:10091000CB09E6E6FAE40E94FF2411F00C94F404FB
:100920000091D000013011F00C9498040E94D90A73
:10093000A4EBB0E04D915C91A8EBB0E00D911C915F
:100940000417150718F011F00C94F2040027A1ED1C
:10095000B0E08C9184FB0EF401E040E0041711F04C
:100960000C94C504E8EBF0E0FA93EA935A924A92A9
:1009700080E0A42DB52D8C9381E00E9482220E94FC
:10098000E40B249681E00E947E220027A1EDB0E0D6
:100990008C9184FB0EF401E041E0041711F00C94FB
:1009A000F2040E94F50A0027A1EDB0E08C9184FBCF
:1009B0000EF401E040E0041711F00C94F204E8EBAF
:1009C000F0E0FA93EA935A924A9280E0A42DB52D72
:1009D0008C9381E00E9482220E94E40B249681E0A5
:1009E0000E947E220C94CB09EEE6FAE40E94FF24DA
:1009F00011F00C9402050E94D90A80E08093C60091
:100A00000C94CB09E0E7FAE40E94FF2411F00C9467
:100A10003E050091D000013011F00C943C050027F8
:100A2000ABE6B0E08C9181FB0EF401E040E00417EE
:100A300011F00C942C058EB5887F8EBD89B78B7F05
:100A400089BF80916B00826080936B0084E690E0A8
:100A50000E94A7230C943C0580916B008D7F8093AE
:100A60006B0080E29EE490934D0080934C0081E007
:100A70008EBD89B7846089BF0C94CB09E8E6FAE49F
:100A80000E94FF2411F00C94D6050091D000013093
:100A900011F00C944D050E94D90AA8EBB0E00E9419
:100AA00095220027A1EDB0E08C9183FB0EF401E0CC
:100AB00041E0041711F00C9472050027ABE6B0E09A
:100AC0008C9182FB0EF401E040E0041711F00C94CD
:100AD0006D05A8EBB0E00E949C228091D100877F39
:100AE0008093D100A4EBB0E04D915C91A8EBB0E015
:100AF0000D911C910417150718F011F00C94820544
:100B00000C94880581E090E0A8EBB0E08D939C9375
:100B10000027A1EDB0E08C9184FB0EF401E040E0F1
:100B2000041711F00C94A705E8EBF0E0FA93EA93B0
:100B30005A924A9280E0A42DB52D8C9381E00E94B8
:100B400082220E94E40B249681E00E947E220027EC
:100B5000A1EDB0E08C9184FB0EF401E041E00417BC
:100B600011F00C94D4050E94F50A0027A1EDB0E025
:100B70008C9184FB0EF401E040E0041711F00C941A
:100B8000D405E8EBF0E0FA93EA935A924A9280E0B7
:100B9000A42DB52D8C9381E00E9482220E94E40B4B
:100BA000249681E00E947E220C94CB09E2E7FAE4CD
:100BB0000E94FF2411F00C944E060091D0000130E9
:100BC00011F00C94E5050E94D90AA8EBB0E00D9154
:100BD0001C91013050E0150718F011F00C94F2054B
:100BE0000C94F805A8EBB0E00E949C220C9400063F
:100BF000A4EBB0E08D919C91A8EBB0E08D939C9319
:100C00000027A1EDB0E08C9184FB0EF401E040E000
:100C1000041711F00C941F06E8EBF0E0FA93EA9346
:100C20005A924A9280E0A42DB52D8C9381E00E94C7
:100C300082220E94E40B249681E00E947E220027FB
:100C4000A1EDB0E08C9184FB0EF401E041E00417CB
:100C500011F00C944C060E94F50A0027A1EDB0E0BB
:100C60008C9184FB0EF401E040E0041711F00C9429
:100C70004C06E8EBF0E0FA93EA935A924A9280E04D
:100C8000A42DB52D8C9381E00E9482220E94E40B5A
:100C9000249681E00E947E220C94CB09E4E7FAE4DA
:100CA0000E94FF2411F00C94C106A8EBB0E00E9452
:100CB0009522A4EBB0E04D915C91A8EBB0E00D91D2
:100CC0001C910417150718F011F00C9469060C9488
:100CD0006F0681E090E0A8EBB0E08D939C938EB519
:100CE000887F8EBDA4E7B0E00D911D912D913C91C0
:100CF000A4E9B0E00D931D932D933C930027A1ED43
:100D0000B0E08C9184FB0EF401E040E0041711F098
:100D10000C94B7065A924A92A4E9B0E00D911D9145
:100D20002D913C91A42DB52D0D931D932D933C93A6
:100D300084E00E9482225A924A92A8EBB0E08D9100
:100D40009C91A42DB52D8D939C9382E00E948222CC
:100D50005A924A9280E0A42DB52D8C9381E00E9496
:100D600082220E94200F269687E00E947E22009118
:100D7000D000013011F00C94BF0681E08EBD0C94C0
:100D8000CB09E6E7FAE40E94FF2411F00C94350742
:100D9000A8EBB0E00D911C91013050E0150718F060
:100DA00011F00C94D5060C94DB06A8EBB0E00E9481
:100DB0009C220C94E306A4EBB0E08D919C91A8EBEF
:100DC000B0E08D939C938EB5887F8EBDA4E7B0E094
:100DD0000D911D912D913C91A4E9B0E00D931D93CF
:100DE0002D933C930027A1EDB0E08C9184FB0EF491
:100DF00001E040E0041711F00C942B075A924A923C
:100E0000A4E9B0E00D911D912D913C91A42DB52D3B
:100E10000D931D932D933C9384E00E9482225A925D
:100E20004A92A8EBB0E08D919C91A42DB52D8D93A5
:100E30009C9382E00E9482225A924A9280E0A42DE2
:100E4000B52D8C9381E00E9482220E94200F26966D
:100E500087E00E947E220091D000013011F00C94B6
:100E6000330781E08EBD0C94CB09E8E7FAE40E94D9
:100E7000FF2411F00C944507ECE0F0E0A8EBB0E0A3
:100E80007BE70E94D6240C94CB09EAE7FAE40E949F
:100E9000FF2411F00C9459078DE181BD85E181BDDE
:100EA0000E94D90A81B5886081BD0C9455070C94C5
:100EB000CB09ADE6B0E0ECE7FAE40E94FF2481E064
:100EC00008F480E08F93ADE6B0E0EEE7FAE40E942C
:100ED000FF2481E010F009F080E09F9189238823AE
:100EE00011F40C942D0889B78B7F89BF8EB5887F4C
:100EF0008EBD0E94F722A0E6B0E08C9300916000C6
:100F0000003011F40C9479070E94FB22A8EBB0E0AA
:100F10008D9388278C9380E08093D00080916B0024
:100F20008D7F80936B00A4EBB0E04D915C91A8EBBA
:100F3000B0E00D911C910417150780E010F009F046
:100F400081E08F93A8EBB0E00D911C91003050E050
:100F5000150781E009F080E09F91892B882311F427
:100F60000C94CD0781E090E0A8EBB0E08D939C93CA
:100F7000E8EBF0E0FA93EA935A924A9281E0A42DCA
:100F8000B52D8C9381E00E9482220E94E40B24966E
:100F900081E00E947E220C942B080027A1EDB0E096
:100FA0008C9184FB0EF401E040E0041781E009F02D
:100FB00080E08F93ADE6B0E0ECE7FAE40E94FF2416
:100FC00081E009F080E09F918923882311F40C943B
:100FD000FC07E8EBF0E0FA93EA935A924A9281E038
:100FE000A42DB52D8C9381E00E9482220E94E40BF7
:100FF000249681E00E947E220027A1EDB0E08C9132
:1010000084FB0EF401E040E0041781E009F080E089
:101010008F93ADE6B0E0EEE7FAE40E94FF2481E0B2
:1010200009F080E09F918923882311F40C942B0808
:10103000E8EBF0E0FA93EA935A924A9280E0A42D0A
:10104000B52D8C9381E00E9482220E94E40B2496AD
:1010500081E00E947E220C94CB09E0E8FAE40E9431
:10106000FF2411F00C9468080E94F722A0E6B0E07B
:101070008C9300916000003011F40C9434080E94AD
:10108000FB22ADEBB0E08C938EB5887F8EBD5A927B
:101090004A928091BD00A42DB52D8C9381E00E94D1
:1010A00082220E94001F229681E00E947E22EBE0B5
:1010B000F0E0ADEBB0E07BE70E94D4240091D000DB
:1010C000013011F00C94660881E08EBD0C94CB09C0
:1010D000E2E8FAE40E94FF2411F00C94B6080E94A2
:1010E000F722A0E6B0E08C9300916000003011F48C
:1010F0000C946F088091C300809360000E94FB22D3
:10110000A3ECB0E08C93A3ECB0E08C918F738C9344
:101110000E942F0B0091C30040E10423A0E6B0E041
:101120000C9300916000003111F00C949B080E9418
:101130002B0B0C949D080E942D0BA3ECB0E08C911E
:101140008F7E8C938EB5887F8EBDEEE0F0E0A3ECB1
:10115000B0E07BE70E94D4240091D000013011F070
:101160000C94B40881E08EBD0C94CB09E4E8FAE459
:101170000E94FF2411F00C941A090091C3004FE360
:101180000423A0E6B0E00C930091D000013011F0F0
:101190000C94CF08A0E6B0E08C9180588C93002787
:1011A000A1EDB0E08C9184FB0EF401E041E0041766
:1011B00011F00C94E008A0E6B0E08C91805C8C9378
:1011C0000027ABE6B0E08C9181FB0EF401E041E03A
:1011D000041711F00C94F108A0E6B0E08C91805E49
:1011E0008C938091B800809362008EB5887F8EBD0D
:1011F00031E0A0E6B0E00E94122331E0ADEBB0E0B8
:101200000E94122331E0A2E6B0E00E9412238091F6
:10121000B4008093620031E0A2E6B0E00E941223A5
:101220000091D000013011F00C94180981E08EBDBE
:101230000C94CB09E6E8FAE40E94FF2411F00C9428
:101240009D09A7EDB0E00D911D912D913C91A3ED6D
:10125000B0E04D915D916D917C910E944624A6E68F
:10126000B0E00D931D932D933D93A6E6B0E00E9450
:101270008622A6E6B0E00D911D912D913C9140E0B3
:1012800052E060E070E00E94C623A6E6B0E00D9355
:101290001D932D933D93A6E6B0E00D911D912D91E8
:1012A0003C91A5ECB0E04C915527662777270E942A
:1012B0002723A6E6B0E04D935D936D937D93A6E65C
:1012C000B0E00D911D912D913C914AE050E060E01D
:1012D00070E00E942723A6E6B0E04D935D936D93E6
:1012E0007D9344E150E060E070E0A6E6B0E00D914F
:1012F0001D912D913C910E944B240CF402C00C9442
:101300008B0900E010E020E030E0A6E6B0E00D93AD
:101310001D932D933C938EB5887F8EBD34E0A6E659
:10132000B0E00E9412230091D000013011F00C9423
:101330009B0981E08EBD0C94CB09E8E8FAE40E9499
:10134000FF2411F00C94B5098EB5887F8EBDA6EAF6
:10135000B0E00E9405230091D000013011F00C9400
:10136000B30981E08EBD0C94CB09EAE8FAE40E944F
:10137000FF2411F00C94CB098EB5887F8EBD0E949E
:10138000BC0E0091D000013011F00C94C90981E02D
:101390008EBD0C94CB0981E090E00E94A7230C94B1
:1013A00061020F921F922F923F924F925F927F9213
:1013B000AF92BF920F931F932F933F934F935F93DF
:1013C0006F937F938F939F93AF93BF93CF93DF934D
:1013D000EF93FF938FB78F93F89489B78B7F89BF73
:1013E0008EB5887F8EBD5A924A9280E092E0A42DFD
:1013F000B52D8D939C9382E00E9482220E94FC2155
:10140000229682E00E947E220091DB000A3011F0D9
:101410000C940C0A0E942B0B0E94461B0091DB00CF
:101420000A3011F00C94190A0E942D0B80E0809371
:10143000DB00ABEDB0E08C918F5F8C93A89500271B
:10144000A1EDB0E08C9184FB0EF401E040E00417C4
:1014500011F00C943E0A5A924A9280E092E0A42D38
:10146000B52D8D939C9382E00E9482220E94FC21E4
:10147000229682E00E947E220E94461BA7EDB0E0E9
:101480004D915D916D917C91A3EDB0E00D911D9119
:101490002D913C910E944B2480E00CF481E08F93CD
:1014A0000027A1EDB0E08C9184FB0EF401E040E058
:1014B000041781E009F080E09F918923882311F4CB
:1014C0000C946F0A80E49CE990934D0080934C004B
:1014D00081E08EBD89B7846089BF0C94BB0A80E02F
:1014E0008093D00080916B008D7F80936B00809102
:1014F0006B008B7F80936B000027BB27A3E38C914D
:1015000080FB0EF401E040E0041711F00C948D0A0A
:1015100080916B00846080936B000027A1EDB0E0A8
:101520008C9184FB0EF401E040E0041711F00C9460
:10153000A20AABE6B0E08C9182FBAAEBB0E0882770
:1015400080F98C930091C3004FE70423A1E6B0E03B
:101550000C930E942D0B80E08093C6000027ABE621
:10156000B0E08C9185FB0EF401E041E0041711F02E
:101570000C94BB0ADF988F918FBFFF91EF91DF91A1
:10158000CF91BF91AF919F918F917F916F915F911B
:101590004F913F912F911F910F91BF90AF907F90EE
:1015A0005F904F903F902F901F900F901895F89458
:1015B000FFCF89B78B7F89BF8EB5887F8EBD80E0D6
:1015C0008093D00080916B008D7F80936B0000270B
:1015D000ABE6B0E08C9185FB0EF401E041E004172E
:1015E00011F00C94F40ADF9808956E98C498C59889
:1015F000C7980E942D0BE2E0F0E00E941E23C49ADF
:101600000E94932384E690E00E94A723A8958091EE
:10161000D1008F7E8093D100E0E6F0E0FA93EA9368
:101620000E941218229600916000003011F40C9470
:10163000280B8091D10080618093D10084E690E0F6
:101640000E94A7236E98C498C598C7980C942A0B3B
:101650000E94110E089597980895979A089581E031
:101660000E94B62380916B008B7F80936B0000916A
:10167000C30041E00423A881B9810C93A881B981FA
:101680000C91003011F40C944A0B80916B00846033
:1016900080936B008091D1008F7D8093D100009169
:1016A000C30042E00423A881B9810C93A881B981C9
:1016B0000C91003011F40C94620B8091D100806287
:1016C0008093D1008091D1008F7B8093D1000091D5
:1016D000C30044E00423A881B9810C93A881B98197
:1016E0000C91003011F40C947A0B8091D10080643D
:1016F0008093D1008091D1008F778093D1000091A9
:10170000C30048E00423A881B9810C93A881B98162
:101710000C91003011F40C94920B8091D1008068F0
:101720008093D10080916B00877F80936B00009144
:10173000C30040E20423A881B9810C93A881B98138
:101740000C91003011F40C94AA0B80916B0088600E
:1017500080936B008091D1008B7F8093D1000091AA
:10176000C40041E00423A881B9810C93A881B98108
:101770000C91003011F40C94C20B8091D100846064
:101780008093D1000091C40046E00423A881B98170
:101790000C93A881B9810C9142E00E94EF240C9334
:1017A000A881B9818C918093D2000091D20003303E
:1017B00011F00C94DE0B82E08093D20081E0481A95
:1017C0008827580A2296089582E00E94B62381E075
:1017D0000E94B6238EB5887F8EBD80916B008D7F71
:1017E00080936B00A4E7B0E00D911D912D913C9189
:1017F000A4E9B0E00D931D932D933C935A924A9225
:10180000A4E9B0E00D911D912D913C91A42DB52D31
:101810000D931D932D933C9384E00E9482225A9253
:101820004A92AA85BB858D919C91A42DB52D8D934F
:101830009C9382E00E9482225A924A9280E0A42DD8
:10184000B52D8C9381E00E9482220E94200F269663
:1018500087E00E947E2240E050E060E070E0A0E976
:10186000B0E00D911D912D913C910E944B2411F0FF
:101870000C943C0C0C940B0E0E94B41E5A924A928B
:101880008091BD00A42DB52D8C9381E00E94822211
:101890000E94001F229681E00E947E225A924A9264
:1018A000AEEBB0E08D919C91A42DB52D8D939C93C2
:1018B00082E00E9482220E94981F229682E00E946B
:1018C0007E220027A1EDB0E08C9182FB0EF401E0B6
:1018D00041E0041711F00C94870C5A924A928091BF
:1018E000C000A42DB52D8C9381E00E9482225A92D3
:1018F0004A928091C100A42DB52D8C9381E00E9465
:1019000082220E94591F249682E00E947E22A4E92E
:10191000B0E00D911D912D913C91A3EDB0E00D93A0
:101920001D932D933C93A4E9B0E00D911D912D9151
:101930003C91A0E9B0E04D915D916D917C910E9448
:101940004124A7EDB0E00D931D932D933D9380E0CE
:10195000A881B9818C930E94461B81E090E0AA8106
:10196000BB818D939C93AA81BB810D911C910F3FEC
:1019700051E0150718F011F00C94ED0CAA81BB8111
:10198000AD90BC90A0EEB0E0AA0DBB1D0C910F3F36
:1019900081E009F080E08F93AA81BB81AD90BC907B
:1019A000A1EEB0E0AA0DBB1D0C910F3E80E010F03F
:1019B00009F081E09F918923882311F40C94E60CAF
:1019C00081E0A881B9818C930C94ED0CAA81BB8134
:1019D0000E94952210F40C94B30CA881B9810C914B
:1019E000013011F00C94AB0CAA81BB81AD90BC907E
:1019F000A2EEB0E0AA0DBB1D8C91AA81BB818D9394
:101A000088278C93AA81BB810D911C9140E150E005
:101A10000E94D622AA81BB814D935C9380E1809382
:101A2000C500AA81BB810D911C91013050E01507C2
:101A300011F00C94200D84E08093C5000C94AD0D42
:101A4000023050E0150711F00C942B0D85E08093C7
:101A5000C5000C94AD0D033050E0150711F00C9447
:101A6000360D86E08093C5000C94AD0D043050E037
:101A7000150711F00C94410D87E08093C5000C947C
:101A8000AD0D053050E0150711F00C944C0D88E0B9
:101A90008093C5000C94AD0D063050E0150711F091
:101AA0000C94570D8AE08093C5000C94AD0D07305F
:101AB00050E0150711F00C94620D8CE08093C50086
:101AC0000C94AD0D083050E0150711F00C946D0D1D
:101AD0008EE08093C5000C94AD0D093050E01507E1
:101AE00011F00C94780D80E18093C5000C94AD0D3D
:101AF0000A3050E0150711F00C94830D84E18093B7
:101B0000C5000C94AD0D0B3050E0150711F00C948E
:101B10008E0D88E18093C5000C94AD0D0C3050E023
:101B2000150711F00C94990D8CE18093C5000C946D
:101B3000AD0D0D3050E0150711F00C94A40D80E2AE
:101B40008093C5000C94AD0D0E3050E0150711F0D8
:101B50000C94AD0D88E28093C500A0E9B0E00D9132
:101B60001D912D913C9140E052E060E070E00E94B8
:101B7000C623A6E6B0E00D931D932D933D93A6E6F4
:101B8000B0E00D911D912D913C91A5ECB0E04C91F0
:101B90005527662777270E942723A6E6B0E04D93B6
:101BA0005D936D937D93A6E6B0E00D911D912D910F
:101BB0003C9148EE53E060E070E00E942723A6E6E7
:101BC000B0E04D935D936D937D93AC81BD810C919D
:101BD000003011F00C940B0E0027ABE6B0E08C91B6
:101BE00085FB0EF401E041E0041711F00C94F90DAF
:101BF000DF9A81E08093D00088EC9FEA90934D00BB
:101C000080934C0089B7846089BF81E08EBD85E0F8
:101C100090E00E94A72383E0481A8827580A249658
:101C20000895A895A4E7B0E00D911D912D913C91E8
:101C3000A8E7B0E00D931D932D933C93A4E7B0E08B
:101C40000D911D912D913C91A4E9B0E00D931D9350
:101C50002D933C935A924A92A4E9B0E00D911D91C4
:101C60002D913C91A42DB52D0D931D932D933C9357
:101C700084E00E9482225A924A9280E090E0A42D51
:101C8000B52D8D939C9382E00E9482225A924A92B3
:101C900080E0A42DB52D8C9381E00E9482220E94C9
:101CA000200F269687E00E947E22A895A4EBB0E044
:101CB0000D911C91013050E0150710F00C94870E27
:101CC0005A924A9281E0A42DB52D8C9381E00E9416
:101CD00082220E94F21F229681E00E947E228CE2E4
:101CE00091E00E94A7235A924A9280E0A42DB52D3C
:101CF0008C9381E00E9482220E94F21F229681E052
:101D00000E947E228091D10080618093D100A895AD
:101D1000A4E7B0E00D911D912D913C91A4E9B0E0B4
:101D20000D931D932D933C93A8EBB0E00D911C9166
:101D3000003050E0150781E009F080E08F93A4EBBC
:101D4000B0E04D915C91A8EBB0E00D911C910417AF
:101D5000150780E010F009F081E09F91892B88231E
:101D600011F40C94B90E81E090E0A8EBB0E08D93F3
:101D70009C930E942D0B089584E00E94B623A3ED4E
:101D8000B0E00D911D912D913C91A881B9810D93E9
:101D90001D932D933C93A4E7B0E00D911D912D91DF
:101DA0003C91A4E9B0E00D931D932D933C935A927E
:101DB0004A92A4E9B0E00D911D912D913C91A42D82
:101DC000B52D0D931D932D933C9384E00E948222A8
:101DD0005A924A928FE19EE4A42DB52D8D939C9347
:101DE00082E00E9482225A924A9280E0A42DB52D70
:101DF0008C9381E00E9482220E94200F269687E029
:101E00000E947E22A4E7B0E00D911D912D913C919E
:101E1000A4E9B0E00D931D932D933C93A881B98163
:101E20000D911D912D913C91A3EDB0E00D931D936B
:101E30002D933C9384E0481A8827580A22960895E7
:101E400081E00E94B62381E00E94B62381E00E94D7
:101E5000B62380E090E0A6EBB0E08D939C93809158
:101E60006B008F7E80936B0000E010E020E030E09C
:101E7000A0E9B0E00D931D932D933C930027ABE6B2
:101E8000B0E08C9183FB0EF401E041E0041781E0A7
:101E900009F080E08F93A885B9850D911C910030E1
:101EA00050E0150781E009F480E09F9189238F932A
:101EB000AE81BF810C91003081E009F080E09F91FC
:101EC0008923882311F40C94C00FA8E9B0E0E885B9
:101ED000F9850E945E24E8E9F0E0A8E6B7E00E94F8
:101EE000BA24E8E6F7E0A8E9B0E01127222704E0E9
:101EF00033270E94032481E4AC81BD818C93AC81A3
:101F0000BD818C9180939E0081E0E8E9F0E001E0E2
:101F10000A93ADE6B0E00E94BF24ADE6B0E08C913C
:101F2000AFE9B0E08C9382E0E8E9F0E001E00A93E9
:101F3000ADE6B0E00E94BF24ADE6B0E08C91A0EA2F
:101F4000B0E08C9383E0E8E9F0E001E00A93ADE6CD
:101F5000B0E00E94BF24ADE6B0E08C91A1EAB0E011
:101F60008C9384E0E8E9F0E001E00A93ADE6B0E0AC
:101F70000E94BF24ADE6B0E08C91A2EAB0E08C9361
:101F800089B78B7F89BF8EB5887F8EBD81B588610B
:101F900081BD877F81BDACECB0E00D911D912D918D
:101FA0003C91A8ECB0E00D931D932D933C93A8E7D2
:101FB000B0E04D915D916D917C91A4E7B0E00D9101
:101FC0001D912D913C910E944B2411F00C94F20F25
:101FD00002E010E020E030E0A8ECB0E00D931D93AB
:101FE0002D933C9380E0A881B9818C93EA81FB8199
:101FF000FA93EA935A924A92AE85BF850D911D914C
:102000002D913C91A42DB52D0D931D932D933C93B3
:1020100084E00E9482220E943D1D249684E00E945A
:102020007E22AA81BB810C910E3F11F40C942410E6
:102030008091D10080618093D10080916B0080619C
:1020400080936B000C9437105A924A92AA85BB85F4
:102050008D919C91A42DB52D8D939C9382E00E942F
:1020600082220E943A11229682E00E947E22A8815A
:10207000B9818C918F5F8C9340917100A881B98157
:102080000C91041781E009F080E08F930027ABE604
:10209000B0E08C9184FB0EF401E041E0041781E094
:1020A00009F480E09F918923882311F40C94ED10AA
:1020B000009180000B3011F00C949A10E8ECF0E0E5
:1020C000FA93EA935A924A92A8ECB0E00D911D91CE
:1020D0002D913C91A42DB52D0D931D932D933C93E3
:1020E00084E00E9482220E947A15249684E00E9455
:1020F0007E22EA85FB85FA93EA935A924A92A8ECEB
:10210000B0E00D911D912D913C91A42DB52D0D9315
:102110001D932D933C9384E00E9482220E9410150F
:10212000249684E00E947E2280E0A881B9818C936D
:102130000C94EB10A8E7B0E04D915D916D917C910E
:10214000A4E7B0E00D911D912D913C910E944B248C
:1021500011F00C94B110AA85BB850E9486220C94C4
:10216000EB10E8ECF0E0FA93EA935A924A92A8EC6A
:10217000B0E00D911D912D913C91A42DB52D0D93A5
:102180001D932D933C9384E00E9482220E947A1535
:10219000249684E00E947E22EA85FB85FA93EA93E6
:1021A0005A924A92A8ECB0E00D911D912D913C916C
:1021B000A42DB52D0D931D932D933C9384E00E9487
:1021C00082220E941015249684E00E947E2280E0E4
:1021D000A881B9818C930C94F110AA85BB850E94CB
:1021E00086220027ABE6B0E08C9184FB0EF401E080
:1021F00041E0041711F00C94F60FC49AA885B98534
:102200000D911C91003050E0150711F00C94101145
:10221000A6EBB0E08D919C91A4EBB0E08D939C93E4
:102220000091D000013081E009F080E08F93002719
:10223000A1EDB0E08C9184FB0EF401E040E00417C6
:1022400081E009F080E09F918923882311F40C94A8
:10225000341180E593EC90934D0080934C0081E025
:102260008EBD89B7846089BF83E0481A8827580AE1
:102270002696089584E00E94B62384E00E94B62347
:1022800081E00E94B62381E00E94B62381E00E9493
:10229000B62381E00E94B62380E0AE81BF818C939B
:1022A000AE81BF810C910F3018F011F00C941D130A
:1022B00081E0AC81BD818C93AC81BD810C910C30EF
:1022C00018F011F00C947C118FEF0E949A230E9459
:1022D0009C230E949B23AC81BD81AD90BB24A2E8CE
:1022E000B0E0AA0DBB1D8C93AC81BD818C918F5F3A
:1022F0008C9310F40C945C118DE0AC81BD818C93B7
:10230000AC81BD810C91043118F011F00C949A113C
:102310008FEF0E949A230E949C230E949B23A881F6
:10232000B9818C93AC81BD818C918F5F8C9310F4BB
:102330000C948011EA85FB85FA93EA93EA85FB8584
:10234000FA93EA930E94A51324960027ABE6B0E027
:102350008C9184FB0EF401E041E0041711F00C9421
:10236000B3110C94151380E0AA81BB818C9300916A
:102370008E00003281E009F080E08F9300918E00A2
:10238000003181E009F080E09F91892B882311F4CE
:102390000C94CE1181E0AA81BB818C9300918300C3
:1023A000003081E009F480E08F9300918300053EC6
:1023B00081E009F480E09F9189238F93AA81BB81FA
:1023C0000C91013081E009F080E09F9189238823FE
:1023D00011F40C940A1300918E00003211F00C9449
:1023E000F511A6EBB0E00E9495220027ABE6B0E025
:1023F0008C9183FB0EF401E040E0041711F00C9483
:102400002A1281E0AC81BD818C93AC85BD854D9154
:102410005C91A6EBB0E00D911C910417150781E0CB
:1024200009F080E08F93A6EBB0E00D911C91003095
:1024300050E0150780E010F009F081E09F918923BA
:10244000882311F40C94281280E0AC81BD818C9318
:102450000C945E1280E0AC81BD818C9381E0A881F8
:10246000B9818C93A881B9810C91053018F011F0D5
:102470000C945E12A881B981AD90BB24ADE9B0E0A7
:10248000AA0DBB1D4C91A881B981AD90BB24A2E8D7
:10249000B0E0AA0DBB1D0C91041711F40C94561258
:1024A00081E0AC81BD818C930C945E12A881B981CE
:1024B0008C918F5F8C9310F40C943212AC81BD819F
:1024C0000C91003081E009F080E08F93AC85BD85F0
:1024D0000D911C910F315EE4150781E009F080E059
:1024E0009F91892B882311F40C940A130E943713AF
:1024F000A885B9850D911D912D913C9140E052E048
:1025000060E070E00E942723A0E9B0E04D935D9366
:102510006D937D93E4E9F0E0FA93EA935A924A923C
:10252000AE85BF850D911D912D913C91A42DB52DAA
:102530000D931D932D933C9384E00E9482220E9470
:102540001015249684E00E947E2280918E00809354
:102550008F00AC85BD850D911C910F315EE4150790
:1025600011F00C94DB12A8E6B7E0E6EBF0E00E9475
:102570005E240E940323ECE8FAE40E940B23A6EAFF
:10258000B0E00E940523ECE8FAE40E940B230091DE
:102590008E00003111F00C94D112EEE8FAE40E94A2
:1025A0000B23A8E6B7E0E885F9850E9461240E9424
:1025B00003230E941723AC81BD810C91003011F0E0
:1025C0000C940A1380916B00806180936B000091E2
:1025D0008F00003181E009F080E08F93AC85BD85EC
:1025E0000D911C910F315EE4150781E009F480E044
:1025F0009F918923882311F40C940A13AA85BB8523
:102600000D911D912D913C91ACECB0E00D931D937B
:102610002D933C9300918300003011F00C9415131E
:1026200080916B00806180936B00AE81BF818C9143
:102630008F5F8C9310F40C9450118FEF0E949A23AB
:102640000E949C230E949B23A0E6B0E08C938FEF16
:102650000E949A230E949C230E949B23A0E6B0E044
:102660008C938CE0481A8827580A2C96089581E0AC
:102670000E94B623A6EAB0E088278C9381E0A88167
:10268000B9818C93A881B9810C91083018F011F0B0
:102690000C947113A881B981AD90BB24A2E8B0E07D
:1026A000AA0DBB1D0C91003211F40C946913A88182
:1026B000B981AD90BB24A2E8B0E0AA0DBB1D8C91FE
:1026C000A6EAB0E08F930E94F0228F918D93882725
:1026D0008C93A881B9818C918F5F8C9310F40C94AA
:1026E0004213A6EAB0E00E94F022E2E9FAE40E9476
:1026F000E92389E0A881B9818C93A881B9810C91E3
:102700000B3018F011F00C949F13A881B981AD9093
:10271000BB24A2E8B0E0AA0DBB1D8C91A6EAB0E0F4
:102720008F930E94F0228F918D9388278C93A8819C
:10273000B9818C918F5F8C9310F40C947D1381E0A0
:10274000481A8827580A2296089581E00E94B623E5
:1027500081E00E94B62384E00E94B6238FEF0E949E
:102760009A230E949C230E949B23AC81BD818C9361
:102770008FEF0E949A230E949C230E949B23AA8190
:10278000BB818C93AA81BB810C911127222733270F
:1027900040E051E060E070E00E94C623A885B98562
:1027A0000D931D932D933D93A885B9850D911D9192
:1027B0002D913C91AC81BD814C915527662777279F
:1027C0000E944124A885B9850D931D932D933D93B7
:1027D000A885B9850D911D912D913C9140E050E067
:1027E00061E070E00E94C623A881B9810D931D931A
:1027F0002D933D938FEF0E949A230E949C230E9469
:102800009B23AC81BD818C938FEF0E949A230E9401
:102810009C230E949B23AC81BD818C938FEF0E94EF
:102820009A230E949C230E949B23AC81BD818C93A0
:102830008FEF0E949A230E949C230E949B23AC81CD
:10284000BD818C938FEF0E949A230E949C230E944B
:102850009B23AC81BD818C938FEF0E949A230E94B1
:102860009C230E949B23AA81BB818C93AA81BB815C
:102870000C9111272227332740E051E060E070E0FF
:102880000E94C623A885B9850D931D932D933D9372
:10289000A885B9850D911D912D913C91AC81BD818B
:1028A0004C915527662777270E944124A885B98532
:1028B0000D931D932D933D93A885B9850D911D9181
:1028C0002D913C91A881B9814D915D916D917C9143
:1028D0000E944124A885B9850D931D932D933D93A6
:1028E0008FEF0E949A230E949C230E949B23AC811D
:1028F000BD818C938FEF0E949A230E949C230E949B
:102900009B23AA81BB818C93AA81BB810C91112747
:102910002227332740E051E060E070E00E94C623A8
:10292000A881B9810D931D932D933D93A881B98101
:102930000D911D912D913C91AC81BD814C915527FC
:10294000662777270E944124A881B9810D931D93A2
:102950002D933D938FEF0E949A230E949C230E9407
:102960009B23AC81BD818C938FEF0E949A230E94A0
:102970009C230E949B23AA81BB818C93AA81BB814B
:102980000C9111272227332740E051E060E070E0EE
:102990000E94C623AE81BF810D931D932D933D935D
:1029A000AE81BF810D911D912D913C91AC81BD8176
:1029B0004C915527662777270E944124AE81BF811D
:1029C0000D931D932D933D93AE81BF810D911D916C
:1029D0002D913C9140E050E061E070E00E94C62300
:1029E000AE81BF810D931D932D933D93AE81BF8129
:1029F0000D911D912D913C91A881B9814D915D91D1
:102A00006D917C910E944124AE81BF810D931D93F5
:102A10002D933D9386E0481A8827580A26960895F4
:102A200084E00E94B62384E00E94B623AC81BD817D
:102A30000D911D912D913C9142E050E060E070E0DD
:102A40000E944624A881B9810D931D932D933D9337
:102A5000A1E7B0E00C91112722273327A881B98183
:102A60004D915D916D917C910E94C623AA81BB819D
:102A70000D931D932D933D93AA81BB810D911D91C3
:102A80002D913C91A8E7B0E04D915D916D917C91C5
:102A90000E944124AA81BB810D931D932D933D93E8
:102AA000009180000B3011F40C946815AA81BB8151
:102AB0000D911D912D913C9140E250E060E070E05D
:102AC0000E944124AA81BB810D931D932D933D93B8
:102AD000AA81BB810D911D912D913C91AE81BF8149
:102AE0000D931D932D933C9388E0481A8827580A2C
:102AF0002496089584E00E94B62382E00E94B623C3
:102B0000009180000B3011F00C94BE15AC81BD819A
:102B10000D911D912D913C9140E850E060E070E0F6
:102B20000E942723A3EDB0E04D935D936D937D93B9
:102B3000AC81BD810D911C9140E850E00E94D622ED
:102B4000A881B9810D931C93A881B9810D911C9125
:102B500044E050E00E94BC23A881B9810D931C93EE
:102B6000A881B9810D911C9144E050E0040F151F1C
:102B7000A881B9810D931C930C94F415AC81BD818F
:102B80000D911D912D913C9140E051E060E070E08D
:102B90000E942723A3EDB0E04D935D936D937D9349
:102BA000AC81BD810D911C9140E051E00E94D62284
:102BB000A881B9810D931C93A881B9810D911C91B5
:102BC00042E050E00E94BC23A881B9810D931C9380
:102BD000A881B9810D911C9142E050E0040F151FAE
:102BE000A881B9810D931C93A3EDB0E00D911D91C7
:102BF0002D913C91ACE7B0E04D915D916D917C9150
:102C00000E944124A3EDB0E00D931D932D933D93BD
:102C1000A3EDB0E00D911D912D913C91AFE6B0E098
:102C20004D915C91662777270E944124A3EDB0E087
:102C30000D931D932D933D930E94461BA881B9814E
:102C4000AD90BC90A0EEB0E0AA0DBB1D8C91AA8106
:102C5000BB818D9388278D938D938C93A881B981A7
:102C60000E949C22AA81BB810D911D912D913C91C6
:102C700040E051E060E070E00E94C623AA81BB8181
:102C80000D931D932D933D93AA81BB810D911D91B1
:102C90002D913C91A881B981AD90BC90A0EEB0E09F
:102CA000AA0DBB1D4C915527662777270E9441240A
:102CB000AA81BB810D931D932D933D9300918000BC
:102CC0000B3011F00C94C416A881B9810E949C228B
:102CD000AA81BB810D911D912D913C9140E051E065
:102CE00060E070E00E94C623AA81BB810D931D9312
:102CF0002D933D93AA81BB810D911D912D913C9106
:102D0000A881B981AD90BC90A0EEB0E0AA0DBB1D2A
:102D10004C915527662777270E944124AA81BB81C1
:102D20000D931D932D933D93A881B9810E949C2200
:102D3000AA81BB810D911D912D913C9140E051E004
:102D400060E070E00E94C623AA81BB810D931D93B1
:102D50002D933D93AA81BB810D911D912D913C91A5
:102D6000A881B981AD90BC90A0EEB0E0AA0DBB1DCA
:102D70004C915527662777270E944124AA81BB8161
:102D80000D931D932D933D93AA81BB810D911D91B0
:102D90002D913C91AE81BF810D931D932D933C935A
:102DA00086E0481A8827580A2496089581E00E94F0
:102DB000B62381E00E94B62309B340EF0423AA8121
:102DC000BB810C93AA81BB810C9148E00E94EF2447
:102DD0000C930027BB27A3E38C9184FB0EF401E046
:102DE00041E0041711F00C94FA16AA81BB818C9172
:102DF0008F5F8C93AA81BB818C9180958C93AA81E3
:102E0000BB810C914FE10423AC81BD810C93002761
:102E1000ABE6B0E08C9185FB0EF401E041E00417D5
:102E200011F00C941B17AA81BB810C914FE0042375
:102E3000AC81BD810C9382E0481A8827580A2496F9
:102E4000089581E00E94B62381E0A881B9818C9326
:102E5000AA81BB814C91A881B9810C91041718F00B
:102E600011F00C944E175A924A9282E0A42DB52D7F
:102E70008C9381E00E9482220E94F21F229681E0C0
:102E80000E947E228DE790E00E94A723A881B9814D
:102E90008C918F5F8C9310F40C94281781E0481A62
:102EA0008827580A2296089581E00E94B62381E07F
:102EB000A881B9818C93A881B9810C91063018F052
:102EC00011F00C9477170E942B0B8FE090E00E947A
:102ED000A7230E942D0B84E690E00E94A723A881DF
:102EE000B9818C918F5F8C9310F40C945B1781E007
:102EF000481A8827580A229608950E949323C39A55
:102F000080E991E00E94A72381B5886081BD0E947D
:102F1000B41E5A924A9281E0A42DB52D8C9381E083
:102F20000E9482220E94001F229681E00E947E223F
:102F300081B5886181BD877F81BD88EC90E00E946A
:102F4000A723FF27E0E1FA93EA935A924A928BE093
:102F5000A42DB52D8C9381E00E9482220E948821AD
:102F6000249681E00E947E22013051E0150711F085
:102F70000C94D3175A924A92AEEBB0E08D919C918B
:102F8000A42DB52D8D939C9382E00E9482220E94F5
:102F9000981F229682E00E947E22E4E9FAE40E94D1
:102FA0000B230E9417235A924A9282E3A42DB52D37
:102FB0008C9381E00E9482220E94001F229681E071
:102FC0000E947E22C29AD89A82E390E00E94A723B0
:102FD000089581E00E94B62381E00E94B6238FEF1E
:102FE000AA81BB818C9380E0A881B9818C93A88150
:102FF000B9810C91073018F011F00C940C1891E085
:10300000AA81BB810E948923A881B9818C918F5F9D
:103010008C9310F40C94F71782E0481A8827580A0A
:103020002496089581E00E94B62381E00E94B62391
:1030300081E00E94B62382E00E94B62382E00E94D3
:10304000B6238FEFAA85BB858C9381E0A885B985CF
:103050008C93A885B9850C91003418F011F00C946C
:103060003B180E94E917A885B9858C918F5F8C93D6
:1030700010F40C942918C49881E0A885B9858C9324
:10308000A885B9850C91003418F011F00C945218F1
:103090000E94E917A885B9858C918F5F8C9310F4F5
:1030A0000C9440188AE090E00E94A723A895EE8136
:1030B000FF81FA93EA935A924A9280E4A42DB52DA7
:1030C0008C9381E00E9482225A924A9200E010E0A2
:1030D00020E030E0A42DB52D0D931D932D933C934E
:1030E00084E00E9482220E94231E269685E00E9490
:1030F0007E22AE81BF810C91013011F40C948918AD
:10310000C49AE8E9FAE40E940B230E9417230C9466
:10311000401B81E0AA85BB858C93A89580E090E058
:10312000A881B9818D939C93EE81FF81FA93EA93F4
:103130005A924A9281E4A42DB52D8C9381E00E948D
:1031400082225A924A9200E010E020E030E0A42D62
:10315000B52D0D931D932D933C9384E00E94822204
:103160000E94231E269685E00E947E22A881B981B6
:103170000E949522AE81BF810C91003081E009F060
:1031800080E08F93A881B9810D911C91003050E0AF
:10319000150781E009F080E09F91892B882311F4C5
:1031A0000C949418C49AA881B9810D911C91003097
:1031B00050E0150711F00C94E518E0EAFAE40E94DB
:1031C0000B230E9417230C94401BA89584E690E0E3
:1031D0000E94A723A895C49881E090E00E94A723AD
:1031E000EE81FF81FA93EA935A924A9280E5A42DE8
:1031F000B52D8C9381E00E9482225A924A9201E07E
:1032000010E020E030E0A42DB52D0D931D932D93FB
:103210003C9384E00E9482220E94231E269685E031
:103220000E947E2285E090E00E94A723C49A8AE053
:1032300090E00E94A723A89500E010E020E030E095
:10324000ACE7B0E00D931D932D933C9300E010E0AC
:1032500020E030E0A3EDB0E00D931D932D933C935F
:103260000E94461B00E010E020E030E0A3EDB0E05B
:103270000D931D932D933C930027A1EDB0E08C910D
:1032800084FB0EF401E041E0041711F00C944A199C
:103290000C94401BA8950091ED00023011F40C94A1
:1032A000DE198091A30280938000AAEAB2E00D911A
:1032B000112740E051E00E94BC23AA81BB810D93FD
:1032C0001C93AA81BB810D911C91A9EAB2E04D919A
:1032D0005527040F151FAA81BB810D931C93AA814A
:1032E000BB810D911C912227332740E050E061E023
:1032F00070E00E94C623ACE7B0E00D931D932D93C0
:103300003D93A8EAB2E00D91112740E051E00E9400
:10331000BC23AA81BB810D931C93AA81BB810D9113
:103320001C91A7EAB2E04D915527040F151FAA8101
:10333000BB810D931C93ACE7B0E00D911D912D91D5
:103340003C91AA81BB814D915C91662777270E94B1
:103350004124ACE7B0E00D931D932D933D93009174
:1033600080000C3011F00C94B8198BE08093800031
:10337000009180000E3011F00C94C1198BE0809305
:103380008000009180000F3011F00C94CA198BE07E
:1033900080938000ACE7B0E00D911D912D913C91A0
:1033A000A3EDB0E00D931D932D933C930E94461B1B
:1033B000A3EDB0E00E94A3220C94321A00911701F1
:1033C000063411F00C94081A84E08093800087E39F
:1033D000A885B9858C93A885B9850C910C3318F014
:1033E00011F00C94061AA885B985AD90BB24A0EE07
:1033F000B0E0AA0DBB1D8C910E941A23A885B98547
:103400008C918F5F8C9310F40C94EB190E9417230E
:1034100000913301063411F00C94321A8BE0809342
:10342000800083E5A885B9858C93A885B9850C9122
:10343000073518F011F00C94301AA885B985AD90B5
:10344000BB24A0EEB0E0AA0DBB1D8C910E941A23F4
:10345000A885B9858C918F5F8C9310F40C94151A04
:103460000E941723EAEAFAE40E940B23A8E6B7E0D9
:10347000E0E8F0E00E946D240E9403230E941723DD
:10348000ECEBFAE40E940B23A8E6B7E0ECE7F0E0EF
:103490000E9461240E9403230E94172384E0A885D0
:1034A000B9858C93A885B9850C910B3018F011F073
:1034B0000C946D1AA885B985AD90BB24A0EEB0E040
:1034C000AA0DBB1D8C910E941A23A885B9858C91E9
:1034D0008F5F8C9310F40C94521A0E9417238091E2
:1034E000EE0080937100EEECFAE40E940B23A8E654
:1034F000B7E0E1E7F0E00E946D240E9403230E9400
:10350000172300917100003011F00C94891A0C946B
:10351000401B00917100003418F011F00C94921AC5
:103520000C94941A0C94401B8091EF00AE81BF81E3
:103530008C938091F000AC81BD818C93AC81BD8176
:103540009C91AE81BF818C91AFE6B0E08D939C934E
:103550008091F700AE81BF818C938091F800AC819F
:10356000BD818C93AC81BD819C91AE81BF818C91DA
:10357000A2E7B0E08D939C93A2E7B0E00D911C917F
:10358000003050E0150711F00C94DC1A8091050111
:10359000AE81BF818C9380910601AC81BD818C93FB
:1035A000AC81BD819C91AE81BF818C91A2E7B0E0DE
:1035B0008D939C930C94DC1AA2E7B0E00D911C91C2
:1035C000003050E0150711F00C94E81A0C94401BE1
:1035D00002E010E020E030E0A2E7B0E04D915C9125
:1035E000662777270E94C623A4E7B0E00D931D93BA
:1035F0002D933D93A4E7B0E00D911D912D913C9149
:10360000AFE6B0E04D915C91662777270E94412498
:10361000A4E7B0E00D931D932D933D93A4E7B0E094
:103620000D911D912D913C91A3EDB0E04D915D91D7
:103630006D917C910E944124A4E7B0E00D931D930D
:103640002D933D93EEEDFAE40E940B23A8E6B7E03C
:10365000E4E7F0E00E9461240E9403230E94172304
:10366000A4E7B0E00D911D912D913C91A3EDB0E048
:103670000D931D932D933C9380E0AA85BB858C937D
:1036800087E0481A8827580A2A96089581E00E9400
:10369000B62381E00E94B62382E00E94B62382E036
:1036A0000E94B6238FEFAE81BF818C9391E0AE81F3
:1036B000BF810E94892391E0AE81BF810E9489234E
:1036C00091E0AE81BF810E94892391E0AE81BF81EC
:1036D0000E94892391E0AE81BF810E94892391E0FD
:1036E000AE81BF810E94892391E0AE81BF810E949B
:1036F000892391E0AE81BF810E94892391E0AE8150
:10370000BF810E94892391E0AE81BF810E948923FD
:1037100091E0AE81BF810E94892391E0AE81BF819B
:103720000E94892391E0AE81BF810E94892391E0AC
:10373000AE81BF810E94892391E0AE81BF810E944A
:10374000892391E0AE81BF810E948923C49880E0E3
:1037500090E0A881B9818D939C938FEF0E949A236A
:103760000E949C230E949B23AE81BF818C93A881E1
:10377000B9810E949522AE81BF810C91003081E019
:1037800009F480E08F93A881B9810D911C910030DC
:1037900050E0150781E009F080E09F91892B882394
:1037A00011F40C94AD1BA881B9810D911C910030CE
:1037B00050E0150711F00C94EA1BE6EEFAE40E94C3
:1037C0000B230E9417238091D10080618093D10048
:1037D0000C94371DEE81FF81FA93EA935A924A9234
:1037E00081E5A42DB52D8C9381E00E9482225A920E
:1037F0004A92A3EDB0E00D911D912D913C91A42D25
:10380000B52D0D931D932D933C9384E00E9482224D
:103810000E94231E269685E00E947E220027A1EDAD
:10382000B0E08C9184FB0EF401E041E0041711F04C
:103830000C942A1CE4EFFAE40E940B23A8E6B7E0FC
:10384000E3EDF0E00E9461240E9403230E9417230D
:103850000C94371DA895AE81BF810C91003011F0FA
:103860000C94751C80E090E0A881B9818D939C93A5
:103870008FEF0E949A230E949C230E949B23AE817B
:10388000BF818C93A881B9810E949522AE81BF81AE
:103890000C91003081E009F480E08F93A881B98118
:1038A0000D911C91003050E0150781E009F080E097
:1038B0009F91892B882311F40C94381CA881B9811D
:1038C0000D911C91003050E0150711F00C94751CFF
:1038D000EEE0FBE40E940B230E9417238091D100AD
:1038E00080618093D1000C94371DAE81BF810C9113
:1038F0000F3F11F00C94BF1C80E090E0A881B981CB
:103900008D939C938FEF0E949A230E949C230E9488
:103910009B23AE81BF818C93A881B9810E9495229F
:10392000AE81BF810C910F3F81E009F480E08F935D
:10393000A881B9810D911C91003050E0150781E0FC
:1039400009F080E09F91892B882311F40C94821C4C
:10395000A881B9810D911C91003050E0150711F03C
:103960000C94BF1CECE1FBE40E940B230E94172384
:103970008091D10080618093D1000C94371DAE817D
:10398000BF810C910E3F11F40C94DC1CEAE2FBE4C5
:103990000E940B23A8E6B7E0EE81FF810E946D2410
:1039A0000E9403230E941723C49A8091D100806152
:1039B0008093D1000C94371D80E090E0AA81BB81F8
:1039C0008D939C9380E0AE81BF818C93AE81BF814B
:1039D0000C910F3F18F011F00C941E1DAA81BB81B1
:1039E0000E9495228FEF0E949A230E949C230E949E
:1039F0009B23AA81BB81AD90BC90A0EEB0E0AA0D44
:103A0000BB1D8C93AA81BB810E9495228FEF0E94DF
:103A10009A230E949C230E949B23AA81BB81AD9084
:103A2000BC90A0EEB0E0AA0DBB1D8C93AE81BF810F
:103A30008C918F5F8C9310F40C94E61C8FEF0E9496
:103A40009A230E949C230E949B23AE81BF818C936A
:103A50008FEF0E949A230E949C230E949B23AE8199
:103A6000BF818C93C49AA3EDB0E00E94862286E0C9
:103A7000481A8827580A2896089582E00E94B6239B
:103A800081E00E94B62380E0AE81BF818C930E94CA
:103A9000E917C49880E090E0AA81BB818D939C9344
:103AA0008FEF0E949A230E949C230E949B23A8814F
:103AB000B9818C93AA81BB810E949522A881B9818A
:103AC0000C91003081E009F480E08F93AA81BB81E2
:103AD0000D911C91003050E0150781E009F080E065
:103AE0009F91892B882311F40C94501DAA81BB81CE
:103AF0000D911C91003050E0150711F00C948D1DB4
:103B0000E6EEFAE40E940B230E9417238091D10075
:103B100080618093D1000C941D1EE881F981FA9395
:103B2000EA935A924A9281E5A42DB52D8C9381E0B7
:103B30000E9482225A924A92AA85BB850D911D91BC
:103B40002D913C91A42DB52D0D931D932D933C9358
:103B500084E00E9482220E94231E269685E00E9415
:103B60007E22A881B9810C91003011F00C94E41DE3
:103B700080E090E0AA81BB818D939C938FEF0E949F
:103B80009A230E949C230E949B23A881B9818C9335
:103B9000AA81BB810E949522A881B9810C91003035
:103BA00081E009F480E08F93AA81BB810D911C9183
:103BB000003050E0150781E009F080E09F91892BEB
:103BC000882311F40C94BE1DA881B9810C910F3F7C
:103BD00011F00C94171E80E090E0AA81BB818D93B8
:103BE0009C938FEF0E949A230E949C230E949B2308
:103BF000A881B9818C93AA81BB810E949522A8815A
:103C0000B9810C910F3F81E009F480E08F93AA8184
:103C1000BB810D911C91003050E0150781E009F047
:103C200080E09F91892B882311F40C94F11DA881C9
:103C3000B9818C91AE81BF818C9383E0481A88272B
:103C4000580A2496089584E00E94B62381E00E94D9
:103C5000B62382E00E94B6238FEFAA81BB818C93AA
:103C600091E0AA81BB810E94892391E0A885B98552
:103C70000E948923AE81BF810D911D912D913C91B0
:103C800040E052E060E070E00E94C623AC81BD815C
:103C90000D931D932D933D93AC81BD818F9314960D
:103CA0008E910E94A91E8E910E94A91E8E910E9443
:103CB000A91E8E910E94A91E85E90E94A91E8F91BE
:103CC00080E090E0A881B9818D939C938FEF0E9452
:103CD0009A230E949C230E949B23AA81BB818C93E0
:103CE000A881B9810E949522AA81BB810C910F3FC6
:103CF00081E009F480E08F93A881B9810D911C9136
:103D0000003050E0150781E009F080E09F91892B99
:103D1000882311F40C94661EA881B9810D911C9121
:103D2000003050E0150711F00C94A11EE8E3FBE40D
:103D30000E940B230E9417238091D1008061809301
:103D4000D100AA81BB818C91AA85BB858C930C94F0
:103D5000AE1E8FB9779BFECF8FB1089587E0481ACA
:103D60008827580A269608955A924A9284E298E043
:103D7000A42DB52D8D939C9382E00E9482225A92AD
:103D80004A9280E0A42DB52D8C9381E00E9482227E
:103D90000E942D21249683E00E947E22EF93FF93C0
:103DA000ECE8F1E00E947B23FF91EF91BB27A0E3B9
:103DB0008C9182FBDEF789E190E00E94A7235A9262
:103DC0004A9280E298E0A42DB52D8D939C9382E0D9
:103DD0000E9482225A924A9280E0A42DB52D8C93A3
:103DE00081E00E9482220E942D21249683E00E947D
:103DF0007E2289E190E00E94A7230E94B51F0895CA
:103E000082E00E94B62300E011E0AA81BB814D91BF
:103E100055270E94BC23A881B9810D931C93A881CA
:103E2000B9810D911C91AA81BB814D915527040F39
:103E3000151FA881B9810D931C935A924A92AA81A9
:103E4000BB818D919C91A42DB52D8D939C9382E087
:103E50000E9482225A924A928BE0A42DB52D8C9317
:103E600081E00E9482220E942D21249683E00E94FC
:103E70007E225A924A9280E298E0A42DB52D8D932D
:103E80009C9382E00E9482225A924A9280E0A42D62
:103E9000B52D8C9381E00E9482220E942D212496D0
:103EA00083E00E947E2282E0481A8827580A2296E0
:103EB000089582E00E94B62300E110E0AC81BD814C
:103EC0004D9155270E94BC23A881B9810D931C9365
:103ED000A881B9810D911C91AA81BB814D91552773
:103EE000040F151FA881B9810D931C935A924A9211
:103EF000AA81BB818D919C91A42DB52D8D939C930E
:103F000082E00E9482225A924A9282E0A42DB52D2C
:103F10008C9381E00E9482220E942D21249683E0CE
:103F20000E947E2282E0481A8827580A2296089525
:103F30005A924A92AA81BB818D919C91A42DB52D54
:103F40008D939C9382E00E9482225A924A9283E04F
:103F5000A42DB52D8C9381E00E9482220E942D21F8
:103F6000249683E00E947E22089581E00E94B62379
:103F700081E00E94B623C49AD898C29880E0A881B4
:103F8000B9818C9380E0AA81BB818C93AA81BB818B
:103F90000C910F3118F011F00C94EA1F91E0A881F8
:103FA000B9810E94892391E0A881B9810E94892367
:103FB00091E0A881B9810E94892391E0A881B9810B
:103FC0000E948923AA81BB818C918F5F8C9310F40E
:103FD0000C94C61FC29AD89A82E0481A8827580AB9
:103FE0002496089581E00E94B6235A924A9280E274
:103FF00098E0A42DB52D8D939C9382E00E9482229F
:104000005A924A9280E0A42DB52D8C9381E00E94B3
:1040100082220E942D21249683E00E947E22AA8182
:10402000BB810C91003011F00C9425205A924A92D9
:1040300080E0A42DB52D8C9381E00E9482220E9405
:104040009F20229681E00E947E22AA81BB810C9152
:10405000013011F00C943B205A924A9285E6A42D2F
:10406000B52D8C9381E00E9482220E949F2022968F
:1040700081E00E947E22AA81BB810C91023011F066
:104080000C9468205A924A9283E6A42DB52D8C9305
:1040900081E00E9482220E949F20229681E00E945D
:1040A0007E2288EC90E00E94A7235A924A9280E0F8
:1040B000A42DB52D8C9381E00E9482220E949F2026
:1040C000229681E00E947E2282E390E00E94A72354
:1040D000AA81BB810C91033011F00C9491205A926B
:1040E0004A9282E6A42DB52D8C9381E00E94822213
:1040F0000E949F20229681E00E947E2280E991E02A
:104100000E94A7235A924A9280E0A42DB52D8C9349
:1041100081E00E9482220E949F20229681E00E94DC
:104120007E228AE090E00E94A7238AE090E00E942D
:10413000A72381E0481A8827580A2296089581E02B
:104140000E94B623C49AD898C298AA81BB810C91C8
:10415000003018F011F00C94AF200C94E92083E5A6
:10416000A881B9818C9391E0A881B9810E948923AB
:104170008FEEA881B9818C9391E0A881B9810E94CA
:1041800089238EE6A881B9818C9391E0A881B981B9
:104190000E94892391E0AA81BB810E94892380E04B
:1041A000A881B9818C9391E0A881B9810E9489236B
:1041B00091E0A881B9810E94892391E0A881B98109
:1041C0000E94892391E0A881B9810E9489230C94DF
:1041D000252185E4A881B9818C9391E0A881B981DA
:1041E0000E94892388E7A881B9818C9391E0A881F6
:1041F000B9810E94892389E6A881B9818C9391E0D5
:10420000A881B9810E94892384E7A881B9818C9310
:1042100091E0A881B9810E94892380E0A881B981B9
:104220008C9391E0A881B9810E94892391E0A881B3
:10423000B9810E94892391E0A881B9810E948923D4
:1042400091E0A881B9810E948923C29AD89A81E01D
:10425000481A8827580A2296089581E00E94B623BA
:10426000C29AD8985A924A9282E0A42DB52D8C9386
:1042700081E00E9482220E94E221229681E00E9437
:104280007E225A924A92AC81BD818C91A42DB52D8B
:104290008C9381E00E9482220E94E221229681E09A
:1042A0000E947E22AC81BD8111968C91A881B9813A
:1042B0008C935A924A92AA81BB818C91A42DB52DE0
:1042C0008C9381E00E9482220E94E221229681E06A
:1042D0000E947E22AC81BD818C91A881B9818C9392
:1042E0005A924A92AA81BB818C91A42DB52D8C93B0
:1042F00081E00E9482220E94E221229681E00E94B7
:104300007E22D89A81E0481A8827580A2296089572
:1043100081E00E94B62381E00E94B62382E00E94E1
:10432000B623C29AD8985A924A9283E0A42DB52D0A
:104330008C9381E00E9482220E94E221229681E0F9
:104340000E947E225A924A92A885B9858C91A42D0A
:10435000B52D8C9381E00E9482220E94E221229658
:1043600081E00E947E22EC81FD81FA93EA930E9413
:10437000E8212296EA81FB81FA93EA930E94E821E0
:104380002296D89AAC81BD810D91112740E051E071
:104390000E94BC23A881B9810D931C93A881B98187
:1043A0000D911C91AA81BB814D915527040F151FBA
:1043B000A885B9850D931C9384E0481A8827580A6C
:1043C0002696089591E0A881B9810E9489230895D5
:1043D00081E00E94B62391E0A881B9810E947E23EA
:1043E000A881B9818C91AA81BB818C9381E0481A04
:1043F0008827580A2296089582E00E94B62381E019
:104400000E94B623C49ABB27A0E38C9182FBDEF7FF
:10441000C298AC81BD810D911C91003052E015070E
:1044200011F00C944B2281E090E0AA81BB818D9326
:104430009C9380E0A881B9818C93A881B9810C916B
:104440000F3018F011F00C944922BB27A0E38C9197
:1044500082FBDEF790E2AA81BB81AD90BC90A0EE1A
:10446000B0E0AA0DBB1D0E948923AA81BB810D91DA
:104470001C9140E250E0040F151FAA81BB810D93EF
:104480001C93A881B9818C918F5F8C9310F40C944C
:104490001D220C94772281E090E0AA81BB818D934C
:1044A0009C93AC81BD814D915C91AA81BB810D91A2
:1044B0001C910417150718F011F00C947722BB27F4
:1044C000A0E38C9182FBDEF7C29A91E0AA81BB81C6
:1044D000AD90BC90A0EEB0E0AA0DBB1D0E94892358
:1044E000AA81BB810E94952210F40C945122C29A99
:1044F00083E0481A8827580A24960895481A88277E
:10450000580A0895480E8827581E08950D911D9148
:104510002D913C9181E0080F8827181F281F381F14
:104520003C932E931E930E930895ED91FC91EF5FB3
:10453000FF4FFC93EE930895ED91FC91E150F04014
:10454000FC93EE9308950D911D912D913C91015096
:104550001040204030403C932E931E930E930895BC
:1045600009D00E94BC2300FC10D0089503D01ED0B7
:1045700001F8F9CF0024E89457FF02C009D06894ED
:1045800000F80BD010F80124089502D009D0089546
:10459000509540954F5F5F4F0895E89417FF089539
:1045A000009510950F5F1F4F68940895352F242FA5
:1045B000E894452B11F468940895512F402F00275B
:1045C000112780E1440F551F001F111F021B130B01
:1045D000416018F4020F131F4E7F8A9599F70895D2
:1045E0008F938D918823E9F711978F91089581E03A
:1045F0005F9B8827089588275F9B089500C05F9B75
:10460000FECF8CB10895A8E6B7E08D91882311F014
:1046100011D0FBCF08950E94EF23802D11F00AD016
:10462000FACF08958D9106D03A95E1F708958DE07F
:1046300001D08AE05D9BFECF8CB9089588EE93E0AF
:1046400086D03197D9F7089500FC05D0089530D071
:1046500005D001F8F9CF37D03FD00895842F952F9A
:10466000A62FB72FE894452B462B472B11F46894BF
:104670000895402F512F622F732F002711272227D3
:104680003327F0E2440F551F661F771F001F111FCD
:10469000221F331F081B190B2A0B3B0B416028F408
:1046A000080F191F2A1F3B1F4E7FFA9559F70895CF
:1046B0000024E89477FF02C006D0689400F809D07F
:1046C00010F80124089512D04F5F5F4F6F4F7F4F56
:1046D0000895E89437FF089500951095209530953A
:1046E0000F5F1F4F2F4F3F4F68940895409550958F
:1046F0006095709508953197F1F708950E949A2377
:104700008C910E949C238D939A95D1F70E949B23B4
:1047100008950E949A238D910E949C239A95D9F71F
:104720000E949B230895BF9ABE98C69ABD9A80E5C1
:104730008DB90895089508958FB9779BFECF8FB1F5
:104740000895689462F80895E89462F80895EF93E4
:10475000FF93EE27E82BE92B31F0E0EDF7E03197FE
:10476000F1F70197D1F7FF91EF9108955A924A928C
:10477000480E8827581E08950F92B801469F800161
:10478000479F100D569F100D0F9008950F921F9286
:104790002F92C801D901489F80014A9F90014B9FE9
:1047A000202C499F100D211D321D5A9F202C589FEF
:1047B000100D211D321D599F200D311D689F200DA8
:1047C000311D699F300D789F300D2F901F900F90F5
:1047D00008950E94EF230D920020D9F70895C895FF
:1047E000319600200895819104D08D938823D9F7C4
:1047F0000895813618F08B3708F48F7D089580E393
:104800000EF4839508952E2E3F2E992781918D3297
:1048100009F093958823D1F79A95E22DF32D112372
:1048200061F0091718F011F0101B01C0191B28F0D6
:1048300021F080E28D931A95E9F780818D3219F489
:104840008D93319604C0222311F08BE28D930917CA
:1048500038F031F0091B21F080E38D930A95E9F7D8
:1048600081918D938823E1F7332351F0EA2FFB2FB9
:10487000319633958E9182933A95E1F78EE28C933F
:104880000895040F151F261F371F0895041B150BCD
:10489000260B370B089504171507260737070895C9
:1048A000000F111F221F331F0895009510952095AA
:1048B00030950F5F1F4F2F4F3F4F0895019110818B
:1048C0000EC001911191219130810BC00191108195
:1048D00017FF05C03FEF2FEF04C0008111272227EB
:1048E000332737FF03C0E1DF8DE28D93CF93DF9352
:1048F000CF92DF92EF92AA24BB24CC24DD24EE24B5
:1049000040E2CAE0DD2755E093E38881890F87FD07
:104910009F7083FD907F891B89935A95A9F7C0DF0B
:10492000AA1CBB1CCC1CDD1CEE1C4A9551F7E8945C
:10493000EFE0FF2782910ED0EB30E0F71EF0689495
:104940008A2D0CD088278D93EF90DF90CF90DF9148
:10495000CF910895982F829501D0892F8F70805D17
:1049600026F0803309F4089568948D93089588277C
:104970008D93089581918D938823E1F7089509918E
:104980009191992351F08A95D9F7319781918D931F
:104990000A9519F08823D1F70895E9CFE199FECF60
:1049A000EEBBFFBB3196089591E001C092E07B37EA
:1049B00051F47FB7F894F2DF8D918DBBE29AE19AC2
:1049C0009A95C9F77FBF7727089591E001C092E0DB
:1049D000E5DFE09A8DB38D939A95D1F70895FF9313
:1049E000881BF9E0001FFA9511F4FF910895881FC4
:1049F000841B18F4840F8894F5CF0894F3CF68943F
:104A000001C0E894AF93BF938D9116F0919103C0CC
:104A10000E94EF23902D891718F011F48823A1F735
:104A2000BF91AF9108955069636F4A6220526561EA
:104A30006C6974792D53797320342E3752004545B3
:104A400070726F6D20002C004D4D4320696E6974AB
:104A500020007265747279202E2E2E00445350204F
:104A6000696E697420004F005A00570052004800D8
:104A7000210059004E0050004200580044004500FB
:104A800056004D005300540049004C0020004420C3
:104A900000002E006F6B00004E6F20636172640097
:104AA00042616420636172640000506172746974D1
:104AB000696F6E2074797065203A000050617274DD
:104AC0006974696F6E2073746172743A0000536583
:104AD00063742F636C757374657220203A00526F93
:104AE0006F74203A000052656164206572726F72C3
:104AF0002031000052656164206572726F7220324D
:104B0000206F6E20736563746F723A2000005265E7
:104B10006164206572726F722033000052656164B7
:104B2000206572726F7220340000526561642065E6
:104B300072726F7220350000526561642074696D75
:064B4000656F75740000B2
:00000001FF
